:0800000000008A110A12052814
:06000A005430FE0001303D
:10001000FF0080308A110A1216218A110A128312F7
:100020000313A1007F08A0005630A2000130A300F6
:10003000831203132008A4002108A500FF30A007A5
:10004000031CA10324082504031995280430220762
:10005000A400A501A50D2308A5072408FE00250876
:10006000FF0080308A110A1216218A110A128312A7
:100070000313A7007F08A6002208FE002308FF0044
:1000800080308A110A1216218A110A128312031370
:10009000A900A5007F08A800A40002302207A40040
:1000A000A501A50D2308A5072408FE002508FF00CB
:1000B00080308A110A1216218A110A128312031340
:1000C000A500AB007F08A400AA0083120313260832
:1000D000AA002708AB00FF30A607031CA7032A08C5
:1000E0002B0403198E282808FE002908FF00803001
:1000F0008A110A1203218A110A1283120313AA0019
:10010000240884008313251883172A088000A80A6E
:100110000319A90AA40A0319A50A6528063083123F
:100120000313A2070318A30A18288A110A123729F1
:10013000080083120313B1007F08B0007E08AF00EF
:10014000B2018312031332082F07B30030080318DB
:10015000013EB40031080318013EB5003308FE002B
:100160003408FF0035088A110A1203218A110A1285
:1001700083120313B60036080319C4283608C520B5
:1001800083120313B20AA128080083120313AE00DE
:10019000831203130C1EC828831203132E08831224
:1001A000031399000800831203138C1AD928981C92
:1001B000D328831203131A0883120313AC00AD0172
:1001C00083120313981CE72883120313AD0A8312CA
:1001D00003132D08013A031DF1288312031318128B
:1001E0001816831203132C0808008316031318151E
:1001F000813099001812831203139817181683166A
:10020000031398160800003A03190A29803A0319C3
:10021000112900347E08840083137F188317000897
:1002200008007F088A007E0882000800003A03194F
:100230001E29803A03192829FF0100347E08840012
:1002400083137F1883170008FF00840A0008080042
:100250008A110A121121FD00FE0FFF03FF0A8A1105
:100260000A121121FC007D08FF007C08080083169B
:10027000031386018A110A12F5208A110A128A11C3
:100280000A12D3208A110A1283120313B7008312B1
:10029000031386008312031337088A110A12C5203C
:1002A0008A110A123F290800013400345C340134F9
:0A02B0003834003401340034003407
:00000001FF
